:10000000830100308A0068288C0003088301A8005F
:100010002408A9002508AA009A30831281070B1131
:100020009B0B3D289B0A2128051E3D289B019B0A0E
:100030003C28051E1F283A28180896000D1697011F
:100040003D28170803191428013A031919280B3AF7
:1000500003191C280030051E0130A4000730A5003C
:100060000310A40DA50B30282408A4000310180CBD
:100070002404980004309B00970A990803194E281D
:1000800019080339031D4D288D1E86148D1A8610FC
:100090008D121A188D1603149A0C99030F08031D5C
:1000A0008F03FF309C07031C9D031D081C04031DC8
:1000B0005E28E1309C0001309D000D158312290857
:1000C000A4002A08A500280883008C0E0C0E090045
:1000D0000D3084000E3075200E30840024307520E1
:1000E00083019B2A04068001840A0406031D7228EA
:1000F0000034A600A71B832827088A002608A60A22
:100100000319A70A82008313271883172608A60A53
:1001100084000008080070346F347734653472341A
:1001200069346E346734203475347034003470347C
:100130006F3477346534723469346E346734203404
:1001400064346F3477346E340034283463342934A3
:100150003234303430343134203442346F34623409
:10016000203442346C34693463346B340034723478
:1001700065346D346F3474346534203476343034FF
:100180002E34353400348207003400340034003417
:1001900000340034003400340034003400340034BF
:1001A0000034003400340034820741344234433494
:1001B0004434453446344734483449344A344B3463
:1001C0004C344D344E344F348207613462346334DE
:1001D0006434653466346734683469346A346B3443
:0801E0006C346D346E346F3491
:1002F400A100803EC72901308312C7210330882919
:100304000D1E82290D12160883120800A1000A305E
:100314008F000F08031D8B29A10B89298312080064
:10032400A2009908031D93298D1222089A003430E3
:10033400990083120800A7292108A7002008A00A11
:100344000319A10A79208312B02121088312A7007E
:10035400200879200038031908009E29A20083127E
:1003640086150F3086052208F03986040615061115
:100374000F308605220EF039860406150611023068
:100384008F000F0803190800C329A20083128611E5
:100394000F3086052208F0398604061506110F3041
:1003A4008605220EF03986040615061102308F00E8
:1003B4000F0803190800DA29A3010830A200063047
:1003C400A000F829073083128605220886040A3023
:1003D400A100A10BEB290518FA29A30A8518FA290B
:1003E400A30A0519FA29A30A0310A20DA00BE429F4
:0C03F400230883120800831286011F30CA
:1004000083168500860197010D129B019B0AE1303E
:100410009C0001309D000D110A30900002309200C6
:100420000F3091008D10143094009E019F019501B2
:1004300081129A30831281008B168B170800831269
:100440008611323088210F3086053030860406153B
:100450000611053088210615061102308F000F089D
:10046000031D2F2A06150611053088210F30860539
:1004700086160615061102308F000F08031D3D2A4F
:100480002830C7210830C7210C30C7210630C729C2
:10049000A0008D1C5C2A8D10522A2008712A200889
:1004A00083126E2A1308013A03194D2A133A0319CD
:1004B0004F2A063A0319962A20302002031C782A74
:1004C0008C2A1030502A83127D21992A1430502A08
:1004D00010308312C7212030B0211030C721992A53
:1004E000003083127A21992A8D1420089300992ACA
:1004F0002008023A0319612A013A0319632A053ACE
:100500000319662A0E3A0319682A043A0319702A55
:10051000013A0319702A742A80302002031C962A9B
:10052000A03020020318962A0730A0052008831265
:10053000B021831208008312FD211F227D21B730D4
:10054000A0000030A1009D2140307A21A530A000FC
:100550000030A1009D21FA308821FA3088217D21C8
:100560000D1E032B8312822148220D14032B8312AC
:10057000851D142B950A06147D218B30A0000030B8
:10058000A1009D2184309E0003309F0008308E0022
:100590000D10142B0D1CD82A0D108E0300301F02D5
:1005A0002D3003191E020318D82A2D309E009F01FA
:1005B0008E080319950A1F081E04031D142B03300F
:1005C0009500831206107D219730A0000030A10015
:1005D0009D2107309E009F01142B0D1C142B0D1024
:1005E0002D309E009F0183128519142B8D1D142B15
:1005F0005A309221142B1F081E04031D142B950141
:1006000083127D21142B1508A40004302402031842
:10061000142B03308A001030240703188A0A820042
:10062000B72ACA2AED2AFB2A8D1D1F2B8D111F0800
:100630001E0403191F2B9E0803199F039E030D1D03
:10064000B02A0D118312DE212B23940BB02A143013
:1006500094008D15B02AA0000F3A031D372B110806
:100660000F3A031D352BA101EA2B0230442B110850
:100670000F3A031D402BA101A10A20089100EA2B8B
:1006800090080319462B0330A100EA2B0430442BB9
:1006900000308A001108D420922B920BFE2B0030E0
:1006A0008A001108D420D32B2108A400053024028D
:1006B0000318FE2B03308A006130240703188A0ACE
:1006C0008200A72B482BB72BBE2B4D2B00308A0066
:1006D0001108D420922B00308A001108E420B52B99
:1006E0002108A400053024020318FE2B03308A00E1
:1006F0007D30240703188A0A8200A72B662B6B2BF8
:10070000FE2BFE2B90080319B72B00308A0011082E
:10071000D420B52B92080319FE2B920100308A00D9
:100720001108E42083129221FE2B2108A400053039
:1007300024020318FE2B03308A00A230240703187A
:100740008A0A8200A72BFE2B822BBE2B8A2B0A3013
:1007500090009201920AFE2B0A30D62B90080319C2
:10076000B72B00308A001108D420831292210A305E
:1007700090009201920A0F309100FE2B900803190D
:10078000FE2B9003FE2B12080A3A031DCD2B0030DE
:100790008A001108E42083129221920BFE2B003074
:1007A0008A001108E4208312922102309200FE2B6D
:1007B0002108A400053024020318FE2B03308A0010
:1007C000E530240703188A0A8200A72BAC2BAE2B36
:1007D000BE2BC32B00308A001108C320A4000430B4
:1007E00024020318BB2B03308A00FA3024070318B5
:1007F0008A0A8200542B702B952BD82B8312080069
:02400E00F13F80
:00000001FF
